:020000040000FA
:100000001A226421A5212B28AD0A0B110900053401
:1000100008343D3412340434823407340E3404344A
:10002000813403341034B23466346034B1348F34E4
:1000300043345034003420344F346834363461341F
:10004000633420344C34433420346D346534743498
:1000500065347234003486160130C8002830CC0074
:1000600007218514061BA528C901C90A061F4920B6
:100070000230E320B5210D307E21363049183A3068
:100080007E211730EC210310BF23462107302422A4
:100090003628C90AC9108514491885107221061B13
:1000A0000800C901B5216D212F307E216921CB00C7
:1000B0008521CA00490794001408203003196328D9
:1000C0002B30941B2D308B21941F68289409940A9F
:1000D000B72246213B0E0F39303E8B217B223B0855
:1000E0000F39303E8B2125308B217E222A30C908E2
:1000F00003198B2172216421031D8D28061B5228B0
:100100004A084907323C03198728C90A5228CE30C9
:100110004A02FF3A013EC900522849080319A4289F
:10012000CA074A0888004B08890083168818962851
:10013000081555308900AA308900881483122A30A6
:100140008B217221B52172215128B52175211B30D7
:10015000C3009C227221B5216D2125307E21D8203B
:100160000319A528D520031DA5283630EC218510BC
:100170007321D8200319A528D520031DA5283230C6
:10018000EC2185147321B521C121B7216D211630D1
:100190007E21D8200319D028D520031DD3280C296F
:1001A0001A307E21C4281F30D128FC302D050800CC
:1001B0004818CC0BDD28C80A07216421031D00283C
:1001C000061F002804300B11AE01AD018101C300F0
:1001D0008B168B1705148316051483127521C30B18
:1001E000EE2883160510831205108B130108AC004E
:1001F000AB018316011601128312AB0301082C0612
:100200000319F9282D082C042E308C0008004818FA
:100210008616481C86120800C921C721A301861F23
:100220001D29D6210A22D82128210B30C3000F30E6
:100230002305031DD3282522C428D821FC21D82139
:100240000E22DD21D821E321D62128210F301629C5
:10025000BF01BE01E830BC000330BD00692185212B
:10026000881B3629BC070318BD0A3729BC070C2296
:10027000D821E830BC000330BD000C22E321D62198
:100280002030971B2D308B219713BB222030A400E8
:10029000B701B801B901BA01BB013730840005309C
:1002A000A600333080078019F039801B0F39800297
:1002B000840AA60B5129BA23BB0DBA0DB90DB80D8E
:1002C000B70DA40B4D29080080300605A902A9002E
:1002D00008000130861F003008007E224330861F50
:1002E0004C308B297321752175217E30A700123087
:1002F000A800A80F7929A70F792900348900862141
:10030000031908008B21890A7F29890083160814A4
:10031000831208080800C20AC00B9529C100061AFA
:100320009429C030C521A02141088515AA002A0EB4
:100330009A212A080F3986004818861605150511D6
:100340004230A700A70BA2290034752185110511A1
:1003500003309A2175219E219E2102309A210C3072
:1003600092212830922106309221013092210930C9
:10037000C0000230C521C201FD30A7006630A800D0
:100380007929421A08007E22C12985119629122254
:10039000CB29323013220E22D621DD21D821DD21B6
:1003A000B7227F309800E3217123D9291223D9295C
:1003B000DC2221308C001D30EC291D308C002130D6
:1003C000EC211830DA291D308C001130EC21183066
:1003D000DA2111308C0018308D000430A6000C0892
:1003E00084000008C4000D088400440880008C03C9
:1003F0008D03A60BEF2908001330C300DD21183050
:100400008400C70147159A228000C30A8403C70BE2
:10041000032A08001730FD293F30132A3630132AEB
:100420003230132A2E30A400DD2124088C0017302E
:10043000EC21A32A83162730810010308500D030AC
:100440008600831285010800C300FE21971F292A18
:1004500097130A30C500C7011808C6008022031987
:10046000342A303E8B21602A47185E2A450303193F
:100470005E2A45089D00C50380220319512A180AE7
:10048000C502031C512AC50A8022043C0318512AC4
:10049000C50A80228C220319482A1D084502031927
:1004A0002E2A1D08C500170B592A04304502031CCB
:1004B0005E2A45084602031C662A652A30308B21D5
:1004C000471498030319762A662A7E22C503031966
:1004D000762AC718752A970B752A47187B22C718E2
:1004E000752A03309700960A960A2E2A7E2216084D
:1004F0007E2115087E29C7142E308B2920308B29A8
:100500004508013E8400040C3C3C84000008451C66
:10051000000E9B000F3908008022013ECA000A3CF1
:100520000319CA011B08F0394A048000451C800EDB
:10053000CA080800430882009A22003E03190800F6
:100540008B21C30A9C2A9E309800A201971FAB2AD8
:10055000C423D222A2170310971BB22ABA23980BE6
:10056000AC2A6D2BA21F97130034940198019701B8
:1005700096019501003494011808031900341708F6
:10058000A20097179E309802981FDA2A9809980AB5
:1005900018080319CF2A0310BF23980BCB2AA21FD8
:1005A0000034C423940A0319950A0319960A0319FF
:1005B000970A00342314FF341808031D1D0803197B
:1005C000B52A17081C06A2001D0898077E30031CD8
:1005D000ED2A98020318102BF02A9802031C6D2BA9
:1005E000C92394179C170310B7221830A500121CBA
:1005F000032B1A0895071B0803181B0F96071C08E6
:1006000003181C0F9707BF23930C920C0310A50B24
:10061000F72A971B0D2BBA239803A21F97130034B8
:10062000A314FF341D0803196F2B18080319B52AEA
:1006300017081C06A20097179C17A501C9231A08C2
:1006400092021B08031C1B0F93021C08031C1C0FA7
:100650009402940193019201031C322B0310BF23D7
:100660000130A5001D089802031C3C2B7E30250795
:1006700098070318102B412B7E3025079807031C81
:100680006D2B1830A400920D930DBA23A50D1A08F6
:1006900095021B08031C1B0F96021C08031C1C0F51
:1006A00097021C0DA504251C572B1214622B1A0847
:1006B00095071B0803181B0F96071C0803181C0A34
:1006C00097071210A40B432BA21F94131408970032
:1006D000130896001208950000342315FF34A31563
:1006E000FF3480309C0617081C06A5009401990170
:1006F00018081D020318E3211D0803190034170808
:10070000A20097179C171D0818029D0003198F2B34
:1007100003109C0C9B0C9A0C990C9D0B882BA51F0D
:100720009C2B99099A099B099C09990A03199A0A11
:1007300003199B0A03199C0A190894071A0803183D
:100740001A0F95071B0803181B0F96071C080318A0
:100750001C0F9707A51BB22B031CB22ABF23980FAF
:10076000B22A102B0318AB2AC423D2228030A2064F
:100770009401AB2A940D950D960D970D0800970CDA
:10078000960C950C940C0800940995099609970904
:100790000800170894001608930015089200080036
:02400E00F23F7F
:10420000000000002500200000006D000000750087
:1042100000006E000000700000002000460000005A
:10422000480000006B0048007A00000020003D00BC
:10423000200000003F003F003F003F0000002A0038
:104240006D00610078002A0000003A0020007A002A
:10425000650072006F0069006E00670000002000BA
:10426000610064006A003A002000000031003A005A
:0C4270002000000032003A002000000096
:00000001FF
